:20FFD600E000E000E000E000E000E000E000E000E000E000E000E000E000FD00E000E000EE
:0AFFF600E000E000E000E000E000A1
:20C00000464C094B5420202020005350454349414C50524F472E3F20202000535045432E07
:20C0200050524F47204B4C41523F200050524F4752414D46454C00000000000000414E475A
:20C0400045204B4F443A00000000000000007300204E31202020204E32202020204E332030
:20C0600000492F4F20544553543F00494E47084E4720414B542E3A00555447084E47204189
:20C080004B542E3A0046454C484953544F52494B3F2020202000204D4A554B2000414E543C
:20C0A0002E50524F472E3A000050554D505449443A00000000445249465452414445524925
:20C0C0004E472021212054454D502031204F46465345543A0054454D502032204F464653CB
:20C0E00045543A0073656B006D003F002E0050524F4752414D4D4552494E472020200020F6
:20C100002000DF4320006D696E00204D4544202000205554414E2000500020003000250006
:20C120006800094E445241204B4F443A0000000000000042525954205354520A4D4D454EA0
:20C14000000000004D41524B45524120494E53502E3F20200053540A545449443A000000B5
:20C16000000000000000202020494E47454E204B4F5247005609524D455220534B0A4C4AA8
:20C1800054414E4B004752414E554C4154004449534B415220202000534B0A4C4A45522000
:20C1A0002000564944415245203D20535441525420200046454C20485556520A52454C53DD
:20C1C000452020005354094E4720485556454E20460A5220002020202020202020202020AD
:20C1E00020202020200056415454454E46594C4C4E494E4720200046594C4C4552205641A5
:20C200005454454E2020200044524946544B4C4152202020202020200046454C2046594C1E
:20C220004C4E494E47202020200050524F562050524F4752414D202020200046454C2048C8
:20C2400059445241554C494B202020002020202053544F5050414420202020200046454C07
:20C26000204B4C094D534B5944442020200046454C2053094B4552482E4E495608200046CC
:20C28000454C204B4F5247445249564E494E470046454C2053094B42525954415245202062
:20C2A0000046454C204D4F544F52534B59444420200046454C200A482D534B594444202002
:20C2C00020200046454C2056415454454E545259434B200053544152543D4A412C203F3D8A
:20C2E0004E454A20004C41444441205354414E444152443F20004C41444441205354414E6F
:20C30000444152443F3F00414E54414C2050524F4752414D3A000000204449534B54494476
:20C32000202000000000000000094E445241200A56524947412020200000534B0A4C4A54FA
:20C34000454D503A000000000000004449534B54454D503A000000000000000053455041FD
:20C36000524154494F4E3A000000000000534B0A4C4A5449443A00000000000000004E49C6
:20C380005608204449534B3A000000000000004E49560820534B0A4C4A3A0000000000002D
:20C3A000464C094B54205449443A00000000000000534B0A4C4A4D4544454C000000000063
:20C3C00000004B4C4152200A565249474120202020200050524F4752414D4D2E204B4C4165
:20C3E000523F2000454E474C4953483F202020202020202000444555545343483F20202094
:20C400002020202020004652414E434149533F20202020202020005356454E534B413F209C
:20C42000202020202020200053554F4D493F20202020202020202020004E454445524C4115
:20C440004E44533F2020202020004954414C49414E4F3F20202020202020004E4F52534B1B
:20C460003F2020202020202020202000455350414E4F4C3F20202020202020200044414E19
:0EC48000534B3F202020202020202020200091
:20C4900046414E202020202020005350454349414C2050524F472E3F202000535045432E98
:20C4B0002050524F472E204F4B3F200050524F4752414D204552524F5200000000494E5024
:20C4D000555420434F44453A0000000000007300204E31202020204E32202020204E3320FB
:20C4F00000492F4F20544553543F00494E47084E4720414B542E3A00555447084E472041F5
:20C510004B542E3A004552524F52204D4553534147455320200020534F465420004E4F2E7B
:20C5300050524F473A0000000050554D5054494D453A00000044524946545241444552499E
:20C550004E472021212054454D502031204F46465345543A0054454D502032204F46465336
:20C5700045543A00736563006D003F002E0050524F4752414D4D494E4720202020200020C0
:20C590002000DF4320006D696E002057495448200020572F4F20200050002000300025006F
:20C5B00068004348414E474520434F44453A00000000005455524E204D414348494E45206A
:20C5D0004F4646004D41524B20494E5350454354494F4E3F00494D50554C53452D54494DB4
:20C5F000453A00000000202020204E4F205241434B20200048454154494E4720424F494CC8
:20C6100045522020004752414E554C4553005741534845532020200052494E534553202093
:20C630002000434F4E54494E5545203D205354415254004552524F5220484F4F444D4F5694
:20C65000454D2E00434C4F534520484F4F4420464F522020002020202020202020202020A3
:20C6700020202020200057415445522D46494C4C494E472020200046494C4C53205741546F
:20C690004552202020202000524541445920544F2057415348202020004552524F52204678
:20C6B000494C4C494E4720202000545249414C2050524F4752414D4D4520004552524F525B
:20C6D000204859445241554C494353002020494E5445525255505445442020200045525253
:20C6F0004F5220484F4F44534146455459004552524F522053414645204C4556454C0045CD
:20C7100052524F52205241434B204452495645004552524F522053414645545953572E207B
:20C73000004552524F52204D4F544F5250524F5420004552524F5220535550455248505226
:20C750004F54004552524F5220574154455250524553530053544152543D59455320202050
:20C770003F3D4E4F004C4F4144204445462E56414C5545533F004C4F4144204445462E56B1
:20C79000414C5545533F004E4F2E204F462050524F4752533A000000205741534854494DDC
:20C7B0004520000000000000004348414E4745204F54482E56414C3F200052494E53452D35
:20C7D00054454D503A000000000000574153482D54454D503A0000000000000053455041E0
:20C7F000524154494F4E3A00000000000052494E53452D54494D453A0000000000004C457A
:20C8100056454C20574153483A0000000000004C4556454C20424F494C45523A0000000005
:20C8300046414E54494D453A00000000000000000052494E53452D4147454E54000000008D
:20C85000000046494E4953484544204F54482E56414C0050524F47522E2046494E495348C9
:20C8700045442000454E474C4953483F202020202020202000444555545343483F20202007
:20C890002020202020004652414E434149533F20202020202020005356454E534B413F2008
:20C8B000202020202020200053554F4D493F20202020202020202020004E454445524C4181
:20C8D0004E44533F2020202020004954414C49414E4F3F20202020202020004E4F52534B87
:20C8F0003F2020202020202020202000455350414E4F4C3F20202020202020200044414E85
:0EC91000534B3F2020202020202020202000FC
:20C920004C0E46544552202020005350455A49414C2050524F472E3F2020005350455A2E7F
:20C9400050524F472E204F4B3F20200050524F4752414D4D204645484C45520000434F4427
:20C96000452045494E474542454E3A0000007300204E31202020204E32202020204E3320A8
:20C9800000492F4F20544553543F00494E47084E4720414B542E3A00555447084E47204160
:20C9A0004B542E3A004645484C45524D454C44554E47454E2000414E5A2E50524F472E3A44
:20C9C000000050554D504544415545523A0044524946545241444552494E4720212120548A
:20C9E000454D502031204F46465345543A0054454D502032204F46465345543A0053656B17
:20CA0000006D003F002E0050524F4752414D4D494552554E47202000202000DF4320004DFE
:20CA2000696E00204D4954202000204F484E452000500020003000250068004E45554552BF
:20CA400020434F44453A0000000000005354524F4D2041425354454C4C454E0000494E5328
:20CA6000502E204D41524B4945522E3F2000494D50554C5344415545523A000000000048B3
:20CA80004549545A5420424F494C4552202020004752414E554C41540053500E4C454E20BB
:20CAA0002020004B4C415253500E4C2000574549544552203D205354415254202000464549
:20CAC000484C2E4841554245424557472E20004841554245205343484C49455353454E0046
:20CAE0002020202020202020202020202020202000460E5220574153534552460E4C4C456A
:20CB00004E00460E4C4C54205741535345522020202000424554524945425342455245495B
:20CB2000542020004645484C455220460E4C4C454E20202000564552535543482050524F7B
:20CB40004752414D4D004645484C2E4859445241554C494B2020002050524F4752414D4DA2
:20CB600053544F50502020004645484C2E4B4C454D4D53434855545A004645484C2E534952
:20CB800043482E4E4956454155004648454C2E4B4F5242414E5452494542004645484C2E47
:20CBA000534943482E534348414C54004645484C2E204D4F544F525343482E200046454864
:20CBC0004C200E482D53434855545A2020004645484C2E574153534552445255434B005357
:20CBE000544152543D4A4120203F3D4E45494E005745524B5357455254204C4144454E3FBB
:20CC0000005745524B5357455254204C4144454E3F00414E5A2E2050524F4752414D4D3AAD
:20CC20000000002053500E4C5A4549542000000000000000414E442E574552544520094E7C
:20CC400044524E3F004B4C415253500E4C544D503A000000000053500E4C54454D503A00F2
:20CC60000000000000000041425452454E4E44415545523A000000004B4C415253500E4CD8
:20CC8000444155523A000000004E49562E2053500E4C454E3A00000000004E49562E2042AC
:20CCA0004F494C45523A00000000004C0E4654455244415545523A00000000004B4C41525F
:20CCC00053502E4D49544C000000000000414E44455245205745525445204F4B3F0050525C
:20CCE0004F4752414D2E204645525449473F00454E474C4953483F20202020202020200027
:20CD0000444555545343483F2020202020202020004652414E434149533F2020202020207E
:20CD200020005356454E534B413F20202020202020200053554F4D493F20202020202020CD
:20CD4000202020004E454445524C414E44533F2020202020004954414C49414E4F3F2020E4
:20CD60002020202020004E4F52534B3F2020202020202020202000455350414E4F4C3F2096
:19CD8000202020202020200044414E534B3F2020202020202020202000CA
:20CDB00056454E54494C4552200050524F472E205350454349414C453F200050524F472E49
:20CDD00020535045432E204F4B3F200050524F4752414D4D452045525245555200494E5328
:20CDF0004552455220434F44453A000000007300204E31202020204E32202020204E33204D
:20CE100000492F4F20544553543F00494E47084E4720414B542E3A00555447084E472041CB
:20CE30004B542E3A00414646495343482E2045525245555220004E425245205047522E3A0C
:20CE500000004455520B4520504D503A000044524946545241444552494E472021212054A5
:20CE7000454D502031204F46465345543A0054454D502032204F46465345543A007365636A
:20CE9000006D003F002E0050524F4752414D4D4154494F4E20202000202000DF4320006D79
:20CEB000696E00204156454320002053414E532000500020003000250068004E4F555645FD
:20CED000415520434F44453A00000000455441494E445245204D4143482E000000504F499C
:20CEF0004E54204420494E53504543542E0054454D505320494D50554C533A000000004DAE
:20CF1000495345200D2054454D5020424F552E004752414E554C4553004C41564520202080
:20CF300020200052494E43452020202000434F4E54494E5545203D205354415254004552A9
:20CF5000522E4645524D2E4341504F542020004645524D2E204341504F5420504F555200DD
:20CF7000202020202020202020202020202020200052454D504C495353414745204541556A
:20CF9000200052454D504C49542045415520202020200050520C5445204155204C41564168
:20CFB000474520004552524555522052454D504C4953532E005047522E204558504552491F
:20CFD0004D454E5420004552522E204859445241554C495155450020202020204152520CD8
:20CFF00054202020202020004552522E4341504F5420534543555220004552522E4E4956B9
:20D01000454155205345435552004552522E454E54522E50414E49455220004552522E49C6
:20D030004E54455252205345435552004552522E5345435552204D4F544555520045525235
:20D050002E20534555522053555243482E004552522E20505245535320454155202000530E
:20D07000544152543D4F554920203F3D4E4F4E0056414C2E4445462E205553494E453F2083
:20D090000056414C2E4445462E205553494E453F3F004E4252452044452050524F47522EA8
:20D0B0003A0000204455522E4C41562E20000000000000004348414E47452041555452209A
:20D0D00056414C3F00544D502052494E0F4147453A000000000054454D50204C415641474D
:20D0F000453A00000000004455522E20534550415241543A000000004455522E2052494EFC
:20D110000F4147453A000000004E49562E204C41564147453A00000000004E49562E204247
:20D130004F55494C4C3A00000000004455522E56454E54494C2E3A00000000004147454EB2
:20D15000542052494E0F2E00000000000050520C54204155545245533F20202020005052CE
:20D170004F47522E5445524D494E0B453F2000454E474C4953483F202020202020202000C2
:20D19000444555545343483F2020202020202020004652414E434149533F202020202020EA
:20D1B00020005356454E534B413F20202020202020200053554F4D493F2020202020202039
:20D1D000202020004E454445524C414E44533F2020202020004954414C49414E4F3F202050
:20D1F0002020202020004E4F52534B3F2020202020202020202000455350414E4F4C3F2002
:19D21000202020202020200044414E534B3F202020202020202020200035
:20D24000505548414C4C494E20004552494B4F49534F484A2E3F20202020004F484A454CFB
:20D260004D4F494E5449204F4B3F20004F484A454C4D4156495248452000000000414E4E4A
:20D2800041204B4F4F44493A0000000000007300204E31202020204E32202020204E33204A
:20D2A00000492F4F20544553543F00494E47084E4720414B542E3A00555447084E47204137
:20D2C0004B542E3A0056494B41484953544F52494120202020004F484A454C2E4C4B4D3A7B
:20D2E000000050554D50505541494B3A000044524946545241444552494E4720212120549D
:20D30000454D502031204F46465345543A0054454D502032204F46465345543A0073656BCD
:20D32000006D003F002E004F484A454C4D4F494E5449202020202000202000DF4320004D62
:20D34000494E00202B2020202000202D202020200050002000300025006800564149484405
:20D3600041204B4F4F44493A000000004B41544B414953452056495254410000004B4952C3
:20D380004A41205441524B49535455533F004B09594E4E4953545953494B413A000000489D
:20D3A000555548542E564544454E204C094D4D0052414550455355200050455355202020A6
:20D3C0002020004855554854454C5520004A41544B41203D20535441525420202000564904
:20D3E000524845204B5556554E4C494B45200053554C4A45204B55505520202020202000A8
:20D400002020202020202020202020202020202000564544454E54095954540A20202020B2
:20D42000200054095954090920564554540920202020004B095954540A56414C4D49532079
:20D440002020200056090952092054095954540A20202020004B4F454F484A454C4D4120A2
:20D460002020202020005649524845204859445241554C2E2020005649524845205059534D
:20D4800009595445545459005649524845204B5556554E52414A4120005649524845205429
:20D4A0005552564152414A412000564952484520504553554B4F5249202000564952484522
:20D4C0002054555256414B59544B2E005649524845204D4F4F54544F5249202000564952DD
:20D4E000484520594C494B55554D2E202000564952484520564553495041494E452000532C
:20D50000544152543D202B2020203F3D202D20004C415441412056414B494F3F2020202043
:20D52000004C415441412056414B494F3F3F202020004F484A454C4D49454E204C4B4D3A37
:20D54000000000502D41494B413A000000000000000000004D55555441204D555554203FA8
:20D56000202020200048555548542E4C094D503A000000000000504553554C094D500A54B6
:20D580003A00000000000052454B45455420504F49533A000000000048555548542E4149B6
:20D5A0004B413A000000000000414E5455524920504553553A0000000000414E5455524968
:20D5C0002048555548543A00000000505548414C4C2E41494B413A000000000048555548E5
:20D5E000542E41494E453A0000000000004D5555542056414C4D49533F20202020004F48C5
:20D600004A454C4D412056414C4D49533F2000454E474C4953483F2020202020202020000D
:20D62000444555545343483F2020202020202020004652414E434149533F20202020202055
:20D6400020005356454E534B413F20202020202020200053554F4D493F20202020202020A4
:20D66000202020004E454445524C414E44533F2020202020004954414C49414E4F3F2020BB
:20D680002020202020004E4F52534B3F2020202020202020202000455350414E4F4C3F206D
:19D6A000202020202020200044414E534B3F2020202020202020202000A1
:20D6D00056454E54494C41542000535045432E50524F472E5354414E443F00535045432EE2
:20D6F0002050524F472E204F4B3F200050524F4752414D4D4120464F55540000005741439C
:20D710004854574F4F52443A0000000000007300204E31202020204E32202020204E332065
:20D7300000492F4F20544553543F00494E47084E4720414B542E3A00555447084E472041A2
:20D750004B542E3A00464F5554204D454C44494E47454E20200041414E542E50524F473ABD
:20D770000000504F4D5054494A443A00000044524946545241444552494E4720212120545D
:20D79000454D502031204F46465345543A0054454D502032204F46465345543A0073656341
:20D7B000006D003F002E0050524F4752414D4D4552454E2020202000202000DF4320004DA1
:20D7D000494E00204D4554202000204745454E2000500020003000250068004E4945555748
:20D7F0002E5741434854573A00000000484F4F4644534348414B2E2055495400004E415AE0
:20D81000494348542050554E543F20202000494D504F4C532054494A443A0000000000561B
:20D830004552572E20424F494C455220202020004B4F5252454C53200057415353454E202C
:20D850002020004E4153504F454C202000564552444552203D205354415254202000464F7E
:20D87000555420484F4544534C554954202000534C55495420484F4544202020202020004D
:20D890002020202020202020202020202020202000564F4F522056554C4C454E20202020BC
:20D8B000200056554C54205741544552202020202020004B4C415220562E20574153534519
:20D8D0004E202000464F55542056554C202020202020202000544553542050524F4752412A
:20D8F0004D4D41202000464F5554204F4C49455359535445454D0050524F47522E4F4E44B3
:20D91000455242524F4B2E00464F5554204B4E454C42455645494C2000464F5554205741AF
:20D930005445524E495645415500464F5554204B4F5246414E44522E202000464F555420A3
:20D9500044455552534348414B202000504F4D50204F56455242454C415354200044524F85
:20D970004F474B4F4F4B20424556202020004C4147452057415445524452554B20200053EB
:20D99000544152543D4A412020203F3D4E454500464142522E494E5354454C4C2E3F2020AF
:20D9B00000464142522E494E5354454C4C2E3F3F200041414E542E50524F4752414D2E3A55
:20D9D0000000002057415354494A443A2000000000000000414E44455245204745472E5780
:20D9F000494A5A3F004E4153504F4C54454D503A00000000000057415354454D503A000053
:20DA1000000000000000004E412057415353454E3A000000000000004E4153504F4C5449D2
:20DA30004A443A0000000000004E49562E2057415354414E4B3A000000004E49562E204203
:20DA50004F494C45523A000000000056454E542E2054494A443A0000000000004E415350DF
:20DA70004F454C4D49442E000000000000414E44455245204745472E204F4B3F2000505223
:20DA90004F4752414D2E4B4C4141523F202000454E474C4953483F2020202020202020009F
:20DAB000444555545343483F2020202020202020004652414E434149533F202020202020C1
:20DAD00020005356454E534B413F20202020202020200053554F4D493F2020202020202010
:20DAF000202020004E454445524C414E44533F2020202020004954414C49414E4F3F202027
:20DB10002020202020004E4F52534B3F2020202020202020202000455350414E4F4C3F20D8
:19DB3000202020202020200044414E534B3F20202020202020202020000C
:208D800056454E544F4C4120200050524F47522E205350454349414C453F0046494E4520DB
:208DA00050524F472E535045432E3F004552524F52452050524F4752414D4D4100434F444A
:208DC00049434520494E5055543A000000007300204E31202020204E32202020204E3320A5
:208DE00000492F4F20544553543F00494E47084E4720414B542E3A00555447084E4720413C
:208E00004B542E3A004552524F524520202020202020202020004E522E505247523A0000F9
:208E200000004F524520504F4D50413A000044524946545241444552494E472021212054DA
:208E4000454D502031204F46465345543A0054454D502032204F46465345543A00736563DA
:208E6000006D003F002E0050524F4752414D4D415A494F4E45202000202000DF4320004DDE
:208E8000494E0020434F4E2020002053454E5320005000200030002500680043414D4249F9
:208EA0004120434F442E3A0000000000535045474E49204D41434348494E4100005350490D
:208EC0004120434F4E54524F4C4C4F3F2000542E204420494D50554C534F3A00000000525B
:208EE000495343414C444920424F494C455220004752414E554C4920004C415641202020C6
:208F000020200053434941435155412000434F4E54494E554F203D20535441525400455296
:208F2000522E4D4F56494D204341505520200043484955444920434150552050455220007A
:208F400020202020202020202020202020202020005249454D50494D2E2041435155412025
:208F600020005249454D504945204143515541202020004F4B204C4156414747494F202097
:208F8000202020004552524F5245204C4956454C4C4F20200050524F4752414D4D41205015
:208FA000524F564120004552522E2049445241554C49434120200020202020415252455357
:208FC000544F2020202020004552522E205345435552204341504F20004552522E204C4966
:208FE000562E2053494355522E004552522E4D4F542E43455354454C4C4F004552522E2052
:209000004D4943524F20504F525441004552522E2050524F54455A2E4D4F542E00455252E0
:209020002E2053555252495343414C442E004552522E2050524553532E4143515541005308
:20904000544152543D5349202020203F3D4E4F0050524F4752414D4120424153453F202050
:209060000050524F4752414D4120424153453F3F20004E522E2050524F4752414D4D493AE8
:20908000000000204455522E4C41563A20000000000000005641522E20414C545249205631
:2090A000414C3F200054DF20534349414351554F3A000000000054DF204C41564147474991
:2090C0004F3A00000000004455522E205345504152415A3A000000004455522E5343494145
:2090E0004351554F3A000000004C49562E4C4156414747494F3A000000004C49562E2042E6
:209100004F494C45523A00000000004455522E56454E54494C2E3A00000000004252494C1E
:209120004C49414E542020000000000000414C54524920564F4C4F5249204F4B3F00464978
:209140004E452050524F4752414D4D413F2000454E474C4953483F2020202020202020000E
:20916000444555545343483F2020202020202020004652414E434149533F2020202020205A
:2091800020005356454E534B413F20202020202020200053554F4D493F20202020202020A9
:2091A000202020004E454445524C414E44533F2020202020004954414C49414E4F3F2020C0
:2091C0002020202020004E4F52534B3F2020202020202020202000455350414E4F4C3F2072
:1991E000202020202020200044414E534B3F2020202020202020202000A6
:20800000564946544520202020005350455349414C50524F472E3F20202000535045432EF3
:2080200050524F472E4B4C41523F200050524F4752414D4645494C2020202020004B4F449B
:20804000453A0000000000000000000000007300204E31202020204E32202020204E33206E
:2080600000492F4F20544553543F00494E47084E4720414B542E3A00555447084E472041C9
:208080004B542E3A004645494C484953544F52494B2020202000414E542E50524F472E3A1B
:2080A000000050554D50455449443A00000044524946545241444552494E47202121205483
:2080C000454D502031204F46465345543A0054454D502032204F46465345543A0073656B60
:2080E000006D003F002E0050524F4752414D4D4552494E4720202000202000DF4320006D7D
:20810000696E00204D4544202000205554454E200050002000300025006800454E4452453B
:20812000204B4F44453A0000000000004252595420535452304D4D454E000000004D455227
:208140004B20494E53502E3F202020202000494D50554C535449443A000000000000005622
:2081600041524D455220534B594C4C54414E4B004752414E554C4154005641534B45522061
:20818000202000534B594C4C4552202000564944455245203D2053544152542020004645A4
:2081A000494C2048455454454245562E2020004C554B4B2048455454454E20464F522000FF
:2081C000202020202020202020202020202020200056414E4E46594C4C4E494E47202020A9
:2081E000200046594C4C45522056414E4E2020202020004452494654534B4C415220202048
:20820000202020004645494C204D45442046594C4C494E47005445535450524F4752414D5B
:208220002020202020004645494C204859445241554C2E202020002020202053544F5050A1
:2082400045542020202020004645494C204B4C454D4245534B2E2020004645494C2053490D
:208260004B4B45482E4E495620004645494C204B5552564452562E202020004645494C205E
:2082800053494B4B2E425259542E20004645494C204D4F544F525645524E202000464549CF
:2082A0004C20542E4B2E53494B522E2020004645494C2056414E4E545259434B202000531D
:2082C000544152543D4A412020203F3D4E4549005354442E20564552444945523F202020FA
:2082E000005354442E20564552444945523F3F202000414E54414C4C2050524F4752414D82
:208300003A0000205641534B5449443A2000000000000000454E44524520414E4E45543F50
:208320002020202000534B594C4C4554454D503A0000000000005641534B4554454D503A8F
:2083400000000000000000534550455241534A4F4E3A000000000000534B594C4C45544978
:20836000443A000000000000004E495641205641534B3A000000000000004E495641205321
:208380004B594C4C3A00000000000056494654455449443A0000000000000000544F525287
:2083A000454D494444454C0000000000004F2E4B2E20414E4E45543F2020202020005052BC
:2083C0004F4752414D204F2E4B2E3F20202000454E474C4953483F20202020202020200029
:2083E000444555545343483F2020202020202020004652414E434149533F202020202020E8
:2084000020005356454E534B413F20202020202020200053554F4D493F2020202020202036
:20842000202020004E454445524C414E44533F2020202020004954414C49414E4F3F20204D
:208440002020202020004E4F52534B3F2020202020202020202000455350414E4F4C3F20FF
:19846000202020202020200044414E534B3F202020202020202020200033
:2084800056454E54494C4152200050524F472E2045535045432E3F2020200050524F472E2E
:2084A0002045535045432E204F4B3F004552524F522050524F4752414D41202000494E54D7
:2084C000524F20434F4449474F3A000000007300204E31202020204E32202020204E3320B9
:2084E00000492F4F20544553543F00494E47084E4720414B542E3A00555447084E47204145
:208500004B542E3A004D414E53414A4553204552524F522020004E522E505247523A0000D5
:2085200000004455522E424F4D42413A000044524946545241444552494E472021212054EC
:20854000454D502031204F46465345543A0054454D502032204F46465345543A00736563E3
:20856000006D003F002E0050524F4752414D4D4143494F4E20202000202000DF4320006D03
:20858000696E0020434F4E2020002053494E2020005000200030002500680043414D4249F1
:2085A0004520434F442E3A0000000000415041474152204D415155494E410000004D415260
:2085C00043415220494E53504543432E3F004455522E20494D50554C534F3A000000004354
:2085E000414C454E54414E444F20424F494C52004752414E554C4F20004C4156414E444F10
:2086000020200041434C415241444F2000434F4E54494E5541523D2053544152540045528E
:20862000522E4D4F56494D204341504F544100434552524152204341504F54412020200063
:20864000202020202020202020202020202020200050415241204C4C454E4152204147551B
:208660004100434F4749454E444F2041475541202020005055454445204C4156415220208A
:20868000202020004552524F52204C4C454E41444F2020200050524F4752414D412044456F
:2086A0002054455354004552522E204859445241554C49434120002020494E5445525550B6
:2086C00043494F4E202020004552522E5345435552204341504F5441004552522E4E49569C
:2086E000454C2053454755522E004552522E4D4F562E43414E4153544120004552522E5359
:20870000454E532E20505545525441004552522E204D4F544F522D50524F542E0045525203
:208720002E50524F5445432E5445524D2E004552522E50524553494F4E20414755410053E2
:20874000544152543D53492020203F3D4E4F4E00204441544F5320464142524943413F203C
:2087600000204441544F5320464142524943413F3F004E522E2050524F4752414D413A0057
:20878000000000204455522E4C41563A20000000000000002043414D422E4F54524F53204B
:2087A00056414C3F0054DF2041434C415241444F3A000000000054DF204C415641444F3A8F
:2087C0000000000000000053455041524143494F4E3A0000000000004455522E41434C4150
:2087E0005241444F3A000000004E49562E2054414E5155453A00000000004E49562E204259
:208800004F494C45523A00000000004455522E56454E54494C2E3A000000000050524F441B
:208820002E204252494C4C4F0000000000204F54524F2056414C2E204F4B3F2020002046F2
:20884000494E414C2050524F4752414D413F00454E474C4953483F202020202020202000F3
:20886000444555545343483F2020202020202020004652414E434149533F20202020202063
:2088800020005356454E534B413F20202020202020200053554F4D493F20202020202020B2
:2088A000202020004E454445524C414E44533F2020202020004954414C49414E4F3F2020C9
:2088C0002020202020004E4F52534B3F2020202020202020202000455350414E4F4C3F207B
:1988E000202020202020200044414E534B3F2020202020202020202000AF
:2089000056454E54494C415420005350454349414C50524F472E3F20202000535045432E71
:2089200050524F47204B4C41523F200050524F4752414D46454A4C2020202020004B4F449F
:20894000453A0000000000000000000000007300204E31202020204E32202020204E332065
:2089600000492F4F20544553543F00494E47084E4720414B542E3A00555447084E472041C0
:208980004B542E3A0046454A4C484953544F52494B3F20202000414E542E50524F472E3AF2
:2089A000000050554D50455449443A00000044524946545241444552494E4720212120547A
:2089C000454D502031204F46465345543A0054454D502032204F46465345543A0073656B57
:2089E000006D003F002E0050524F4752414D4D4552494E4720202000202000DF4320006D74
:208A0000696E00204D4544202000205544454E20005000200030002500680041454E445246
:208A200045204B4F44453A0000000000534C554B20535452304D4D454E000000004D4152DF
:208A40004B455220494E53502E3F20202000494D50554C535449443A0000000000000056C2
:208A600041524D455220534B594C4C54414E4B004752414E554C4154005641534B45522058
:208A8000202000534B594C4C4552202000564944455245203D20535441525420200046459B
:208AA0004A4C204841455454454245562E20004C554B4B204845415454454E20464F5200B3
:208AC000202020202020202020202020202020200056414E44500846594C444E494E47209A
:208AE0002000500846594C4445522056414E4E2020200044524946544B4C41522020202062
:208B00002020200046454A4C204D2E2046594C444E494E47005445535450524F4752414D66
:208B200020202020200046454A4C204859445241554C494B2020002020202053544F505051
:208B4000455420202020200046454A4C204B4C454D4245534B2E20200046454A4C20534902
:208B60004B4B4552482E4E49560046454A4C204B555256454452455620200046454A4C20E5
:208B80004430524B4F4E54414B54200046454A4C204D4F544F52564145524E200046454A90
:208BA0004C20542E4B2E53494B522E20200046454A4C2056414E445452594B202020005340
:208BC000544152543D4A412020203F3D4E454A005354442E20564552444945523F202020F0
:208BE000005354442E20564552444945523F3F202000414E54414C2050524F4752414D3A8B
:208C0000000000205641534B4554443A200000000000000041454E44524520305652494791
:208C2000413F202000534B594C4C4554454D503A0000000000005641534B4554454D503A46
:208C40000000000000000053455041524154494F4E3A000000000000534B594C4C45544973
:208C6000443A000000000000004E4956454155205641534B3A00000000004E495645415557
:208C800020534B594C3A000000000056454E54494C2E5449443A00000000000054305252F4
:208CA000454D494444454C0000000000004B4C4152203056524947453F2020202000505268
:208CC0004F4752414D204F2E4B2E3F20202000454E474C4953483F20202020202020200020
:208CE000444555545343483F2020202020202020004652414E434149533F202020202020DF
:208D000020005356454E534B413F20202020202020200053554F4D493F202020202020202D
:208D2000202020004E454445524C414E44533F2020202020004954414C49414E4F3F202044
:208D40002020202020004E4F52534B3F2020202020202020202000455350414E4F4C3F20F6
:198D6000202020202020200044414E534B3F20202020202020202020002A
:20B0000018CE6002BD96BFBD96BF18CE6002181D00A0181C00408630BD95668630BD956657
:20B020008630BD95668620BD95668628BD9623BD96BF8606BD9623BD96BF8614BD9623BD2D
:1BB0400096BF860CBD9623BD96BF8601BD9623BD96BF18CE6002181C002039A2
:20FF000001010A141E28323C46505152535455565758595A0001010A141E28323C3D3E3F92
:20FF200040414243444546000A141E28323C000A0F14191E23282D32373C0000010F14195C
:1BFF40001E23282D3C4B5AFF000000010300010600000300020300000000FF1E
:20FD0000DD6ADF6C18DF6E132C02107F0038BDECFD2608BDED032603152C02132C400B7CF1
:20FD200000569656810F2E0D20177A0056965681002702200C132C4005152C402003142C85
:20FD400040132C010EBDEC7A7C0068966881072E07200B7F00682006BDECF6152C01132BFC
:20FD600020037C0039132B40037C003A132B10037C00387C00017C003F860A913F2E331363
:20FD8000298005DE3308DF337C0055142A107C00357C00377C00427C0043132B8007DC3BAE
:20FDA000C30001DD3B7C00367F003F132B02037C0054964027087A00402603152A049641E2
:17FDC00027087A00412603152A088640B71025DC6ADE6C18DE6E3BF1
:20E000008600B710248693B710397F10358683B71026863EB710098E00FF8600B760018677
:20E02000FFB760008604B760018600B7600386E0B760028604B76003BD958518CE01F4BDF6
:20E040009533BDF8CC861497BB7F000E7F00217F0022BDF9BEBDF2D7BDF8CCBDFA7CBDEB67
:20E0600056BDEB28BDEEADB6103181FF27037EE084BDEEDFB6103281FF27037EE084BDF8DC
:20E08000CC7EA14486009704BD9651BDED152700BDED032706152A407EA0007EE2C5152ACB
:20E0A00041BD9651CCC09DBDF027DC1BBDEF2EBD9673CCC0A9BDF027DC1DBDEF2ECCC1205E
:20E0C000BDF027BD9822122801F9122804F5BD9651B6B7159767B6B71497669708CCC0C6FB
:20E0E000BDF1859766CEB714BD97EF96679708CCC0D5BDF1859767CEB715BD97EF18CE0122
:20E10000F4BD9533BD9651BD9673CCC050BDF0278681BD9695BDED8D9607BDEF11CCC11A45
:20E12000BDF0278687BD9695BDEDC59607BDEF11CCC11ABDF027868DBD9695BDEDFD960793
:20E14000BDEF11CCC11ABDF027BDE782962D27037EE6BFBDED03262520B6BD9651CCC061F2
:20E16000BDF027BD9673CCC2D4BDF027BD98221228010A122804067E941B7EE25D142C01A4
:20E18000BD9679CCC085BDF027BD9673CCC2D4BDF027BD9822122801E1122804DDBD967958
:20E1A000CCC1D5BDF027BD9679CEB7E0A600BDEF11CCC0ECBDF027CEB7E0A601BDEF11CCB4
:20E1C000C0ECBDF027CEB7E0A602BDEF11CCC0ECBDF027CEB7E0A603BDEF11CCC0ECBDF0B9
:20E1E00027CEB7E0A604BDEF11BD9822BD9679CCC1D5BDF027BD9679CEB7E0A605BDEF111A
:20E20000CCC0ECBDF027CEB7E0A606BDEF11CCC0ECBDF027CEB7E0A607BDEF11CCC0ECBD94
:20E22000F027CEB7E0A608BDEF11CCC0ECBDF027CEB7E0A609BDEF11BD9822BD9679CCC10A
:20E24000D5BDF027BD9679CCC144BDF027BD982212280109122804058663BDF3CABD96519F
:20E26000CCC22ABDF027BD9673CCC2D4BDF027BD9822122801081228040486019704BD96A5
:20E2800079CCC1D5BDF027BD9679CCC155BDF0279603BDEF11BD98221228020F7C00038630
:20E2A0001591032ED98601970320D3BD9679CCC01BBDF027BD982212280107122804037EDB
:20E2C000F6617EE09EBDFA7C142A40BDF8CCBD9651960F972E9610972F152A03152A01BD00
:20E2E000EA61962D27037EE6BFBDED8D2646152A30BD9679CCC1C4BDF027BD9673CCC1E687
:20E30000BDF027BD9822122801F9BDEAC88602912D27D68601912D27C3142A30BD9651BDCE
:20E320009673CCC1F7BDF027142A32BDE99A8601912D27A8142A0386019721142A307F004B
:20E3400033142C04142980BD9673CCC208BDF027BD9822122801F91228040D7EE387BDEAD4
:20E3600061962D27227EE75ABDED1B260DBDEAC8962D27037EE6BF7EE33EBDEA61962D2769
:20E38000037EE6BF7EE33E152C80152C04142A30BD9673CCC1D5BDF027BD9673CCC118BD20
:20E3A000F0279621810027339621BDEF11CCC11ABDF027BDE7019657BDEF11CCC106BDF036
:20E3C00027CCC11ABDF027963081002714963081022708CCC185BDF0272006CCC096BDF0C6
:20E3E00027CC0000DD33142C08142980BD9822122804131228022E7C0021961191212C873A
:20E40000860197212081BDED1B260DBDEAC8962D27037EE6BF7EE387BDEA61962D27037E4A
:20E42000E6BF7EE387152C081529804F91212600BD9673CCC1D5BDF027142A30142C80BD3A
:20E44000EC737F00337F0034142980BDE782962D27037EE6BFCC000F1A93332EEE86009711
:20E46000009701BDE782962D27037EE6BFBDA265BDA284BDE701BDEAC8962D27037EE6BF03
:20E4800018CE07D0BD9544BDE99A962D27037EE387CC0000DD3396698100270D18CE01F4A9
:20E4A000BD9533BDEC3C7EE4C7BDEC657EE4C7BDE782962D27037EE6BFBDF07BCC000E1A40
:20E4C00093332EEBBDECA4BDE782962D27037EE6BFBDF07BCC000F1A93332EEB966981005E
:20E4E0002710BDECA418CE0190BD9533BDEC467EE4FC18CE01F4BD9533BDEC3C18CE0064C0
:20E50000BD9533CCC18EDD58142A80BDE782962D27037EE6BF18CE0190BD9533BDF07BCC42
:20E52000001E1A93332EE44F91302709966981002703BDEC5EBDE782962D27037EE6BFBDE7
:20E54000F07BCC001BD3311A93332EE9BDECDABDE782962D27037EE6BFBDF07BCC001BD3D3
:20E5600031D3641A93332EE7152980BDECB818CE01F4BD953318CE01F4BD9533BDECA418FA
:20E58000CE01F4BD9533BDECE1BDEE712615BD9673CCC1D5BDF027152A80BD9673CCC174D0
:20E5A000BDF027BDE782962D27037EE6BF7A002F7A002FBDEE71270220087C002F7C002F3C
:20E5C00020E17C002F7C002F18CE01F4BD9533BDEC6C18CE01F4BD9533BDEC54142980CC89
:20E5E000C198DD58142A80BDE782962D27037EE6BFDC62C3001BD331D3641A93332EE8BD8F
:20E60000ECC6BD958518CE01F4BD9533BDECE818CE01F4BD9533BDECEFDC151A83000027D3
:20E6200025CCC000DD58BDEC4DBDE782962D27037EE6BFDC62C30028D331D364D3151A93CF
:20E64000332EE6BDECBF960481012727152980152A80BD9673CCC1D5BDF027BD95857F00D2
:20E66000337F0034142A30152C80BDF108BDEA617EE387BDF108BD9673CCC1D5BDF027BD70
:20E680009585152A80BDEA61BD9651152AB0CCC18EDD58CCC22ABDF0271429807F00337F3C
:20E6A0000034BDE782962D27037EE6BFBDED032608CC02321A93332EE9BD96517EE4308662
:20E6C00001912D26037EE2DC8602912D26037EE2E98607912D26037EE387860A912D26038B
:20E6E0007EE2C5860B912D26037EF494860C912D26037EE09E860D912D26037EF1BC7EECF3
:20E700000DB6B7059713B6B70397129621C6033DC3007F8FA600973008A60097579707C6BC
:20E72000B73DDD31BDA2A19613C6033DDD64D331DD5A9612C6033DDD62D35ADD5A96144968
:20E740008102270BC6033DDD15D35ADD5A2005CC000020F3C30028DD5A39BD9679BD9673B7
:20E76000CCC24CBDF02718CE01F4BD9533BD9673CCC1D5BDF02718CE01F4BD9533BDEB285F
:20E7800020D8BD9679BDEFCC132C04037EF412132C08037EF42E132A2007132A1003BDEF29
:20E7A00041132A0126BDEDFD261E860F91422E1BBD9679152A30CCC26EBDF0278605BDF3D2
:20E7C000CA152A01BDE75A397F0042BDED1B2743BDED032745122B0148142B10860A9138C1
:20E7E0002E4CBDEB56BDEB28142B01BDEB28152A80BDED1B2603152A0C142A30BD9651BDFA
:20E80000EA61152B01132A01058607972D398601972D39BDED51270920B6BDECFD27092024
:20E82000B4BDED87270220A8152B107F0038BDED872720BDED3F271B142B20860091392E7B
:20E8400018BD9673CCC27FBDF0278606BDF3CABDEB7E39152B207F00397A002EBDEDFD2706
:20E8600018BDEE3526137C002E7A002E7A002EBDEE35260DBDEC1920087C002EBDEC81207C
:20E88000067C002E7C002E7A002FBDEDC52722BDEE71261D7C002F7A002F7A002FBDEE7145
:20E8A0002617BDED692612BDED81260DBDEC2020087C002FBDEC8820067C002F7C002FBD6C
:20E8C000ED1B271DBDED572718142B40865B913A2E15CCC290BDF0278607BDF3CABDEAAFEF
:20E8E00039152B407F003ABDED6F2720BDED29271B122B0817142B08BD9651CCC2A1DD4995
:20E90000BDF0278608BDF3CABDEBA339BDED21271B122B0417142B04BD9651CCC2B2DD49E5
:20E92000BDF0278609BDF3CABDEBA339132A0217BDED812612BDEDC5260D142B80CC044C40
:20E940001A933B2E11201A152B807F003B122B0227BDEC9D202DBDEC357F0054142B0220D1
:20E9600022BDEC9DBD9651CCC2C3DD49BDF027860ABDF3CABDEBA339860691542E05152BCE
:20E980000220CEBDED51270B863D91362E0BBDEC8F20067F00367F002D397F003DBDE782BD
:20E9A000962D270139BDEDFD2709BDED8D27047F002D39BDEE35261B7A002F7A002FBDEEF7
:20E9C0007127087C002F7C002F20087C002F7C002F20CABDEDC527C5BDE782962D27013934
:20E9E000122B02F47F003718CE03E8BD9533BDEC5496172703BDEC6CBDE782962D270139A5
:20EA00009637815B2E1BBDED8D27ED7F0055BDE782962D270139BDED8D27DD861991552EAD
:20EA2000EDBDECC6BDECE8BD9585BD9673CCC1F7BDF0277C003D860A913D2E22BDEDFD27BF
:20EA40000B8619913D2E17BDED8D2612BD9679CCC219BDF0278602BDF3CABDEBBA397EE93F
:20EA60009D132A2007132A1003BDEF41BDE782962D270139122A04E9122A08E57F0035BD4B
:20EA8000E782962D7F002D270139BDED312607BDEC967F002D39BDEC8FBDEC2E86069135B0
:20EAA0002EDDBDED372711863D91352ED22009BDEB28BDEB567EE75ABD9679CCC23BBDF0B1
:20EAC000278603BDF3CA20E7BDED1B2610BDEC27BDE782962D270139BDED1B271D18CE07FA
:20EAE000D0BD95337F002D39BDE782962D270139862F91362EF27F002D39BDED372617866D
:20EB00004E91362ECBBD9651CCC1B3BDF0278601BDF3CA7EEAAFBD9673CCC25DBDF027860C
:20EB200004BDF3CABDEBE239BDEC9DBDECDABDECA4BDECC6BDEC81BDEC88BDEC96BDEC8F3D
:20EB4000BDECEFBDECBFBDECE1BDECE8BDECB8BDECF6152A80397F00337F00347F003B7F04
:20EB6000003C7F003D7F003E7F00397F003B7F0028152980152A3C152BF0152C0C39BDEB30
:20EB800056BDEB28BDEA61BD9822122801F9122804F5BD9651122A01058602972D39860771
:20EBA000972D39BDEB56BDEB28BDEA61152A03BD9679DC49BDF0277EE75ABDEB56BDEB28EE
:20EBC000BDEA61152A33BD9673CCC1A2BDF027BD9822122801F9122804F5BD965186019752
:20EBE0002D39BDEB56142B01BDEB28152B01BDEA61BD9822122801F9122804F5BD965112C4
:20EC00002A01058602972D398607972D39BD9679CCC02CBDF0277EE75ACE60001C00083913
:20EC2000CE60001C000439CE60001C000239CE60001C000139CE10081C000239CE10081C05
:20EC40000004142A0439CE10081C001039CE10081C000839CE10081C0020142A0839CE1028
:20EC6000001C008039CE10001C004039CE10001C002039CE10001C001039CE10001C0008B4
:20EC800039CE60001D000839CE60001D000439CE60001D000239CE60001D000139CE100836
:20ECA0001D000239CE10081D0004122B0109865B97419740142A0439CE10081D001039CE89
:20ECC00010081D000839CE10081D0020122B0109865B97419740142A0839CE10001D0080CA
:20ECE00039CE10001D004039CE10001D002039CE10001D001039CE10001D000839B660027B
:20ED0000841039B66002840839B66002840439B66002840239B66002840139B6100A8480EF
:20ED200039B6100A8440884039B6100A8420882039B61000840439B610008402880239B664
:20ED40001000840139B66000840839B66000840439B66000840239B66000840139B61000C4
:20ED6000844039B61000842039B61008840239B61008840439B61008841039B610088408E2
:20ED800039B61008842039B610008410398603B7103018CE0001BD9533CE10301E0080055F
:20EDA00086019724397F0024F6103486C43DCE0032028FCE000A028F17970791192E038664
:20EDC00000398601398602B7103018CE0001BD9533CE10301E00800586019724397F002480
:20EDE000F6103386C43DCE0032028FCE000A028F179707911A2E038600398601398604B708
:20EE0000103018CE0001BD9533CE10301E00800586019724397F0024F6103186C43DCE00EB
:20EE200032028FCE000A028F17970791192E038600398601398600B7103018CE0001BD95E1
:20EE400033CE10301E00800586019724397F0024F61031C02C86413DCE0095028FCE0001C6
:20EE6000028F17800A9B66912E2E038600398601398601B7103018CE0001BD9533CE1030F8
:20EE80001E00800586019724397F0024F61032C02C86413DCE0095028FCE0001028F17809E
:20EEA0000A9B67912F2E038600398601398600B7103018CE0001BD9533CE10301E0080053C
:20EEC00086019724397F0024F61031C02C86413DCE0095028FCE0001028FC00ADB663986CF
:20EEE00001B7103018CE0001BD9533CE10301E00800586019724397F0024F61032C02C8635
:20EF0000413DCE0095028FCE0001028FC00ADB673997747F0073BD97438620BD9794CE00EA
:20EF200079A60081202704BD96AF390820F3DD73BD97438620BD9794CE007920E4BD96AFCE
:20EF400039132A2079BDED452704132C4017BD96798681BD9695BDEEAD17BDEF11CCC1027C
:20EF6000BDF0272014BD96798681BD9695CCC0FFBDF027CCC0FFBDF027BDED4B2704132CB1
:20EF80004014868BBD9695BDEEDF17BDEF11CCC102BDF0272011868BBD9695CCC0FFBDF001
:20EFA00027CCC0FFBDF027132C80148687BD9695CCC118BDF0279621BDEF11152A10398608
:20EFC00087BD9695CCC0FFBDF02720EF132A8056BD9673DC58BDF027DC5A93330C59490CBD
:20EFE00059490C59490C59490C5949CE0064028FDD5CCE003C028FD75E863C3DDD5FDC5C26
:20F00000935FD761965EBDEF11CCC0E8BDF027966181092E06CCC11CBDF0279661BDEF11E7
:20F02000CCC0E4BDF0273983C000D3458FBD96AF393C183C3637BD9673CCC11EBDF02720CC
:20F040000CC61086104A26FD5A26F82005BDED0327FB3332183838393C183C3736BD965198
:20F06000CCC11EBDF0273233183838393C183C3736BDED0327FB323318383839BD9679BD70
:20F0800096739633BDEF2E398600CEB709BD97EF8600CEB70908BD97EF8600CEB711BD9765
:20F0A000EF8600CEB71108BD97EF8600CEB713BD97EF8600CEB716BD97EF8600BDF3CA86AF
:20F0C00000BDF3CA8600BDF3CA8600BDF3CA8600BDF3CA8600BDF3CA8600BDF3CA8600BD73
:20F0E000F3CA8600BDF3CA8600BDF3CA8603CEB721BD97EF8608CEB722BD97EFBD9651CCF9
:20F10000C0B5BDF0277EF105B6B7169720FCB709DD1BFCB711DD1DB6B713971F9B57813BA2
:20F120002E56971FDC1BC30001DD1B96209B13813B2E02200C803C9720961F8B01971F9666
:20F14000209720961FCEB713BD97EF9620CEB716BD97EFDC1DCEB711BD97EFDC1D17CEB74D
:20F160001108BD97EFDC1BCEB709BD97EFDC1B17CEB70908BD97EF39803C971FDC1DC3001D
:20F1800001DD1D209FDD49BD9679DC49BDF027960881092E06CCC11ABDF0279608BDEF1198
:20F1A000BD98221228021296088B01970881142E0220D48601970820CE960839152A40BDE1
:20F1C000FA7CBD9679BD9673CCC0FFBDF027BDECFD2708CCC0ECBDF0272003BDF2CDBDED5E
:20F1E000032708CCC0ECBDF0272003BDF2CDBDED092708CCC0ECBDF0272003BDF2CDBDED7B
:20F200000F2708CCC0ECBDF0272003BDF2CDBDED152708CCC0ECBDF0272003BDF2CDBDED42
:20F220001B2708CCC0ECBDF0272003BDF2CDBDED212708CCC0ECBDF0272003BDF2CDBDED0A
:20F24000292708CCC0ECBDF0272003BDF2CDBDED312708CCC0ECBDF0272003BDF2CDBDEDCC
:20F26000372708CCC0ECBDF0272003BDF2CDBDED3F2708CCC0ECBDF0272003BDF2CD868133
:20F28000BD9695BDED8D9607BDEF11CCC11ABDF0278687BD9695BDEDC59607BDEF11CCC12F
:20F2A0001ABDF027868DBD9695BDEDFD9607BDEF11CCC11ABDF027BDED0326037EF1C2BD25
:20F2C000ED0326FBBD96517E926F7EF2BFCCC11CBDF027397EF38E9618970586099706BDE3
:20F2E000F3BC26F09611970586099706BDF3BC26E396109705865A9706BDF3BC26D6960F99
:20F30000970586469706BDF3BC26C996139705863C9706BDF3BC267696139705863C97063D
:20F32000BDF3BC266996129705863C9706BDF3BC265C96199705865A9706BDF3BC264F9602
:20F340001A9705865A9706BDF3BC264296149705865A9706BDF3BC263596179705860197B5
:20F3600006BDF3BC26289666970586149706BDF3BC261B9667970586149706BDF3BC260EE1
:20F380009603970586159706BDF3BC260139BDFA30860A97669767BDF93B9666CEB714BD7F
:20F3A00097EF9667CEB715BD97EF86039718CEB706BD97EF8662BDF3CA7EE75A9605910694
:20F3C00022022003860139860039CEB7E0E600BD97EF0817E600BD97EF0817E600BD97EF49
:20F3E0000817E600BD97EF0817E600BD97EF0817E600BD97EF0817E600BD97EF0817E600E8
:20F40000BD97EF0817E600BD97EF0817E600BD97EF39CC003E1A93332E11BDB000BD967384
:20F42000CCC208BDF027CC0000DD337EE796CC003E1A93332EF5BDB000152C80142A30BD25
:20F440009673CCC1D5BDF027BD9673CCC118BDF02796219621BDEF11CCC11ABDF027BDE7E4
:20F46000019657BDEF11CCC106BDF027CCC11ABDF027963081002714963081022708CCC178
:20F4800085BDF0272006CCC096BDF027CC0000DD337EF42BBD9673CCC2D4BDF027BDFA7C4F
:20F4A000152A027F000EBD9679BDF767BD982212280208BDF776BDF8CC20D9BDF8CCBD9664
:20F4C00073CCC2D4BDF027BD9679CCC2E5BDF027BD98221228011E1228041ABD9679CCC2EE
:20F4E000F6BDF027BD98221228010A12280406BDFA307EF6787C000EBD9679CCC1D5BDF00A
:20F5000027BD9679CCC2F6DD47BDF694BD982212280205BDF77620E086019721BD9679CC50
:20F52000C118BDF0279621BDEF118603D6213DC3007FC30000DD0A8FA60081FF260486009C
:20F54000A7008100270C81022710CCC10ABDF0272029CCC111BDF0272021CCC096BDF02739
:20F56000CCC0FFBDF027CCC0FFBDF027CCC0FFBDF027CCC0FFBDF0277EF581CCC185BDF05C
:20F5800027BD982212280210DE0A6C008603A10026026F00DF0A2084BD9679CCC118BDF0C1
:20F5A000279621BDEF11CCC318BDF0278603D6213DC3007FC30001DD0A8FA60081FF2604AC
:20F5C0008601A700BDEF11CCC106BDF027BD982212280210DE0A6C008609A1002ABA860127
:20F5E000A70020B47C002196118B01912127037EF51C7C000EBD9651BD9673CCC2D4BDF052
:20F6000027BD9679CCC329BDF027BD98221228016712280463BD9679CCC1D5BDF027BD965C
:20F6200079CCC318DD47BDF694BD982212280205BDF77620E97C000E8609910E2AD77F001C
:20F640000EBD9679CCC00ABDF027BD9673CCC2D4BDF027BD982212280107122804037EE012
:20F660009EBD9679CCC3C2BDF027BD9822122802078602970E7EF61EBD9679CCC3D3BDF0A7
:20F6800027BD9822122802037EF494BDF93BBD96517EE2C5BD9673CCC2D4BDF027BD967905
:20F6A0008611D60E3DD347BDF0278601910E26059611BDEF118602910E260B9610BDEF1134
:20F6C000CCC102BDF0278603910E260B960FBDEF11CCC102BDF0278604910E260B9613BDE9
:20F6E000EF11CCC04EBDF0278605910E260B9612BDEF11CCC04EBDF0278606910E261196F6
:20F7000019BDEF11CCC11EBDF027CCC0FFBDF0278607910E2611961ABDEF11CCC11EBDF00D
:20F7200027CCC0FFBDF0278608910E262196144981022712BDEF11CCC04EBDF027CCC0FF2A
:20F74000BDF0277EF74ECCC11CBDF02720E98609910E261296172708CCC10ABDF0272006B9
:20F76000CCC111BDF02739BD96798611D6183DC3C3E4BDF027398600910E26127C0018BD2B
:20F78000F8CC860991182A6F7F00187EF8C88601910E26107C0011860991112A5A86019743
:20F7A000117EF8C88602910E26237F0044CCFF008FD6443AA600810026067F00447F001074
:20F7C00091102E057C004420E49710202A8603910E26277F0044CCFF158FD6443AA600817E
:20F7E0000026067F00447F000F910F2E057C004420E4970F7EF8C87EF8C88604910E262460
:20F800007F0044CCFF288FD6443AA600810026067F00137F004491132E057C004420E49775
:20F82000137EF8C88605910E26237F0044CCFF2F8FD6443AA600810026067F00447F0012BD
:20F8400091122E057C004420E49712207B8606910E261296198B0A9719866391192A697FCE
:20F8600000197EF8C88607910E2612961A8B0A971A8663911A2A517F001A7EF8C8860891D2
:20F880000E26237F0044CCFF3B8FD6443AA60081FF26067F00447F001491142E057C004425
:20F8A00020E4971420228609910E260F961727057F0017201386019717200DCCC02CBDF08B
:20F8C0002718CE03E8BD9533BDFA7239961881002607CCC490DD45202181012607CCC92006
:20F8E000DD45201681022607CCCDB0DD45200B81032607CCC000DD45204081042607CCD25B
:20F9000040DD45203581052607CCD6D0DD45202A81062607CC8D80DD45201F81072607CC30
:20F920008000DD45201481082607CC8480DD45200981092605CC8900DD45399603CEB6D0CE
:20F94000BD97EF960FCEB700BD97EF9610CEB701BD97EF9611CEB702BD97EF9612CEB703E7
:20F96000BD97EF9613CEB705BD97EF9618CEB706BD97EF9619CEB707BD97EF961ACEB71788
:20F98000BD97EF9614CEB719BD97EF9617CEB720BD97EF961BCEB709BD97EF961DCEB71139
:20F9A000BD97EFBDFA72C600CEB60018CE007F18A600BD97EF0818085CD12326F239B6B7F5
:20F9C00000970FB6B7019710B6B7029711B6B7039712B6B7059713B6B7069718B6B70797F3
:20F9E00019B6B717971AB6B7199714B6B7209717FCB709DD1BFCB711DD1DB6B713971FB6EF
:20FA0000B7149766B6B7159767B6B7169720B6B6D09703BDF2D7BDFA72C600CEB60018CEAF
:20FA2000007FA60018A7000818085CD12326F33986059703863C970F8655971086049711D7
:20FA400086149712861E971386289719860A971A8601971486009717BDFA72C600CEFF480C
:20FA600018CE007FA60018A7000818085CD12326F3398603D6113DCB03D7233918CE012C31
:20FA8000BD95337F002C18CE1024181C0040BDEB56152BFF152A80142C40860097560E1893
:04FAA000CE00C83993
:209200008682BD9695BDEEAD4F1BBDEF11CCC102BDF027CCC11ABDF027868ABD9695BDEE5E
:20922000DF4F1BBDEF11CCC102BDF027CCC11ABDF027BD967386C2BD9695BDED8D9607BDC3
:20924000EF11CCC11ABDF02786C7BD9695BDEDC59607BDEF11CCC11ABDF02786CCBD9695E0
:20926000BDEDFD9607BDEF11CCC11ABDF02739BD9200BD9382BDEC3518CE0190BD9533BD81
:20928000EC9DBD9200BD9382BDEC5E18CE0190BD9533BDECDABD9200BD9382BDEC6518CE89
:2092A0000190BD9533BDECE1BD9200BD9382BDEC6C18CE0190BD9533BDECE8BD9200BD93AC
:2092C00082BDEC1918CE0190BD9533BDEC81BD9200BD9382BDEC2018CE0190BD9533BDEC95
:2092E00088BD9200BD9382BDEC2E18CE0190BD9533BDEC96BD9200BD9382BDEC2718CE01DB
:2093000090BD9533BDEC8FBD9200BD9382BDEC7318CE0190BD9533BDECEFBD9200BD93820E
:20932000BDEC4D18CE0190BD9533BDECBFBD9200BD9382BDEC3C18CE0190BD9533BDECA484
:20934000BD9200BD9382BDEC5418CE0190BD9533BDECC6BD9200BD9382BDEC4618CE0190FD
:20936000BD9533BDECB8BD9200BD9382BDEC7A18CE0190BD9533BDECF6BD9200BD93827E89
:20938000926FBDECFD2606BDEC9D7E9390BDEC35BDED032606BDECDA7E939EBDEC5EBDED79
:2093A000092606BDECE17E93ACBDEC65BDED0F2606BDECE87E93BABDEC6CBDED152606BD25
:2093C000EC817E93C8BDEC19BDED1B2606BDEC887E93D6BDEC20BDED212606BDEC967E936C
:2093E000E4BDEC2EBDED292606BDEC8F7E93F2BDEC27BDED312606BDECEF7E9400BDEC73DB
:20940000BDED372606BDECBF7E940EBDEC4DBDED3F2604BDECA439BDEC3C39BDEAC8BDEDF1
:209420001B27F8BD96518600970CBDEC19BD94D4BDEC81BD94CCBDEC20BD94D4BDEC88BD1B
:2094400094CC7C000CBDEC2EBD94D4BDEC96BD94CCBDEC35BD94D4BDEC9DBD94CCBDEC3C81
:20946000BD94D4BDECA4BD94CCBDEC46BD94D4BDECB8BD94CCBDEC4DBD94D4BDECBFBD94F7
:20948000CCBDEC54BD94D4BDECC6BD94CCBDEC5EBD94D4BDECDABD94CCBDEC65BD94D4BD96
:2094A000ECE1BD94CCBDEC6CBD94D4BDECE8BD94CCBDEC73BD94D4BDECEFBD94CCBDEC7AC1
:2094C000BD94D4BDECF6BD94CC7E942618CE03E8BD953339BD9673CCC078BDF0277C000CBE
:2094E000960CBDEF11CCC0FFBDF027BD94F2BD94CC39BDECFD2703142C01BDED0327031419
:209500002C01BDED092703142C01BDED0F2703142C01BDED152703142C01BDED3127031499
:209520002C01BDED372603142C01BDED3F2703142C0139183C3CCE01470926FD38180926D5
:20954000F4183839183C3CCE01470926FD38180926F418383936B66000840F97093284F09B
:209560009A09B760003918CE6002181D0040BD955518CE6002181C0080181D0080181C00AF
:2095800040BD96BF3918CE6002BD96BFBD96BF18CE6002181D00A0181C00408630BD9566D5
:2095A0008630BD95668630BD95668620BD95668628BD9623BD96BF8606BD9623BD96BF86A1
:2095C00014BD9623BD96BF860CBD9623BD96BF8601BD9623BD96BF18CE6002181C00201812
:2095E000CE6002181D0020181D00408640BD9623BD96BF18CE6002181C0020CE9703DF49F7
:2096000086409707DE49A60008DF49BD9623BD96BF96074A9707810026EA18CE6002181CCF
:2096200000203918CE6002970D84F0BD9555BD9640960D840F48484848BD9555BD9640396E
:20964000181D0040181C0080181D0080181C00403918CE6002181D00208601BD9623BD9692
:20966000BFBD96BF18CE6002181C0020398680BD96953986C0BD96953918CE6002181D0039
:20968000208602BD9623BD96BFBD96BF18CE6002181C00203918CE6002181D0020BD9623A0
:2096A000BD96BFBD96BF18CE6002181C002039A600270BBD96230886194A26FD20F13918ED
:2096C000CE0014BD95333936375F8164251A5C8064816424F9CB303617BD9623325F8100E8
:2096E00026068630BD96234F810A250F5C800A810A24F9CB303617BD9623328B30BD962355
:2097000033323904000E111F1111000A000E111F1111000A000E1111110E0003041F101E30
:20972000101F0002051F101E101F0003041F111F1111001100111111111F000E111010103C
:20974000150E037F00707F00717F007286109776CE007286039775A6009777840F80052BA4
:209760000696778B039777967784F080502B0696778B3097779677A700097A007526D878C0
:2097800000747900737900727900717900707A007626BD39CE0079A700088C007D26F8CEB4
:2097A00000009670840F27058B309779089671444444442606D679C12027058B30977A089E
:2097C0009671840F2606D67AC12027058B30977B089672444444442606D67BC12027048B65
:2097E00030977C9672840F8B30977D7F007E3937183CC616F7103BE700C617F7103B18CEF1
:20980000000ABD95337F103BC602F7103BA700C603F7103B18CE000ABD95337F103B1838A4
:20982000333936373C183C152807BDECFD26FBBDED0326F6BDED0926F118CE0019BD95339D
:20984000BDECFD26E5BDED0326E0BDED0926DB132A400ABDE782962D27037EE6BFBD98BD21
:20986000BDECFD27037E988CBDED0327037E9878BDED0927DA7E98A018CE0019BD9533BD66
:20988000ED0327CB142802142C02202818CE0019BD9533BDECFD27B7142801142C02201463
:2098A00018CE0019BD9533BDED0927A3142804142C022000142C01183838333239132A2041
:0998C00007132A1003BDEF413922
:20A00000BDA10DBD96518600970CBD9679CCC03DBDF027960CBDEF11BD9673CCC2D4BDF06B
:20A0200027BD982212280107122804037EA0427C000C960C810A27037EA00A8600970C7EF1
:20A04000A00ACC0000DD0ABD9679CCC03DBDF027960CBDEF11DC0ABDEF2EBD9673CCC2D4F3
:20A06000BDF027BD982212280107122804037EA089DC0AC30001DD0A1A83000A27037EA0EB
:20A0800047CC0000DD0A7EA047960CB1B7212617960BB1B72226102007860C972D7EE6BFF8
:20A0A000860B972D7EE6BFBD9651960C8107260ADC0A1A83000226022007860A972D7EE69E
:20A0C000BF8600970CBD9679CCC03DBDF027960CBDEF11BD9673CCC2D4BDF027BD9822124B
:20A0E000280107122804037EA0FD7C000C960C810A27037EA0C58600970C7EA0C5960C81E3
:20A100000926B7BD9651860D972D7EE6BFBDED0326FBBD9679CCC0EEBDF027BD9673CCC2FF
:20A12000D4BDF027CC0000DD33142980DC331A83000A2E05BDECFD27037EA0BABDED032779
:20A14000EB7EA003152A40BD9651CCC122BDF027B6B721BDEF11B6B722BDEF11BD9673CC24
:20A16000C2D4BDF027BD982212280107122804037EA1767EA20CBD96518600970CBD967921
:20A18000CCC03DBDF027960CBDEF11BD9673CCC2D4BDF027BD982212280107122804037E4F
:20A1A000A1B57C000C960C810A27037EA17D8600970C7EA17DCC0000DD0ABD9679CCC03DC1
:20A1C000BDF027960CBDEF11DC0ABDEF2EBD9673CCC2D4BDF027BD98221228010712280499
:20A1E000037EA1FCDC0AC30001DD0A1A83000A27037EA1BACC0000DD0A7EA1BA960CCEB753
:20A2000021BD97EF960BCEB722BD97EFBD9651CCC133BDF0277EA21518CE6002181D00A0C5
:20A22000181C004018CE6002181C002039BDED0F27037F0001BDE782962D27037EE6BF86B6
:20A240003291012E0896004C97007F0001CC00321A93332ED8960081022E0586019769391B
:20A260008600976939BDED0F2614CC001E1A93332EF3BD9651CCC166BDF0277EE75A7F0098
:20A28000017EA22D96698101270B963081022704860497213996308102270139860097699E
:20A2A000399669810027037EA2B286009713861497129669810127013996308100270139EC
:09A2C000860097138614971239E9
:008000017F
